:020000020000FC
:1000000030C0189501C026C006B3002E0F2404FC92
:100010001895BB98C39A00C000C000C00071B39986
:10002000012BC398BB9A04FD01270061F00EF4FC7C
:100030000EC0F5FE1895FF2427BB05E003BF0BE8B3
:1000400002BF02E008BF09BF00E205BF18952AE021
:10005000F5FC2CE0BA98B99800E305BF13BE19BEB1
:1000600018951124222710E2C49AC09ABB9AFF2443
:1000700000E20BBF00E305BF78948895FECF68616E
:1000800066746D616E6E23736F667477617265005E
:00000001FF
